:10000000FFC1FFC1FFC1FFC1FFC1FFC1FFC1FFC1F0
:10001000FFC1FFC1FFC1FFC1FFC1FFC1FFC1FFC1E0
:10002000FFC1FFC1FFC1FFFFFFFFFFFFFFFFFFFF9A
:10003000FFFFFFFFFFFFFFFFFFFFFFFFFFFFFFFFD0
:10004000FFFFFFFFFFFFFFFFFFFFFFFFFFFFFFFFC0
:10005000FFFFFFFFFFFFFFFFFFFFFFFFFFFFFFFFB0
:10006000FFFFFFFFFFFFFFFFFFFFFFFFFFFFFFFFA0
:10042000FFC1FFC1FFC1FFFFFFFFFFFFFFFFFFFF96
:10043000FFFFFFFFFFFFFFFFFFFFFFFFFFFFFFFFCC
:10044000FFFFFFFFFFFFFFFFFFFFFFFFFFFFFFFFBC
:10045000FFFFFFFFFFFFFFFFFFFFFFFFFFFFFFFFAC
:10046000FFFFFFFFFFFFFFFFFFFFFFFFFFFFFFFF9C
:10082000FFC1FFC1FFC1FFFFFFFFFFFFFFFFFFFF92
:10083000FFFFFFFFFFFFFFFFFFFFFFFFFFFFFFFFC8
:10084000FFFFFFFFFFFFFFFFFFFFFFFFFFFFFFFFB8
:10085000FFFFFFFFFFFFFFFFFFFFFFFFFFFFFFFFA8
:10086000FFFFFFFFFFFFFFFFFFFFFFFFFFFFFFFF98
:100C000039C16DC152C151C150C14FC14EC14DC159
:100C10004CC14BC14AC149C148C147C146C145C188
:100C200044C143C142C105010906A10175019508EE
:100C3000050719E029E715002501810295017508CE
:100C40008103950575010508190129059102950192
:100C500075039103950675081500256505071900AC
:100C600029658100C00902220001010080320904C7
:100C700000000103010100092101010001223F00E0
:100C80000705810308000A12011001000000084254
:100C90004231E10001010200011A03740069006E93
:100CA00000790055005300420062006F006100723D
:100CB000006400520368007400740070003A002F52
:100CC000002F006D006100740072006900780073ED
:100CD0000074006F0072006D002E0063006F006DE5
:100CE000002F006100760072002F00740069006E12
:100CF00000790075007300620062006F006100728D
:100D00000064002F000403090474696E795553428E
:100D1000626F6172640A687474703A2F2F6D617427
:100D200072697873746F726D2E636F6D2F61767256
:100D30002F74696E79757362626F6172642F0A0A2B
:100D40000A496E206361736520796F7520656E6353
:100D50006F757465722070726F626C656D732C2094
:100D60006861766520616E79207175657374696F4D
:100D70006E73206F7220696E20636173650A796FEC
:100D800075206A75737420686176652072656D617F
:100D9000726B732C20706C6561736520646F206EBC
:100DA0006F7420686573697461746520746F206363
:100DB0006F6E746163743A0A5374657068616E2073
:100DC00042616572776F6C6620202D2073746570A8
:100DD00068616E406D617472697873746F726D2EA4
:100DE000636F6D0A6D617472697873746F726D40B0
:100DF000676D782E64652C206F722073746570683F
:100E0000616E2E62616572776F6C664074752D69D4
:100E10006C6D656E61752E64650A0A5047502D4BE6
:100E200065794944093A20307846423942313244A2
:100E3000420A46696E6765727072696E74093A207B
:100E4000323235322042343145203132444620346A
:100E50003141442034373646203746333620303847
:100E60003441203039313120464239422031324438
:100E7000420A000011241FBECFE5D4E0DEBFCDBF83
:100E800010E0A0E6B0E0EAECF7E102C005900D92B8
:100E9000A636B107D9F720E0A6E6B0E001C01D9262
:100EA000AA3AB207E1F723D28EC4AACEA82FB92F4F
:100EB00080E090E041E050EA609530E009C02D917B
:100EC00082279795879510F084279527305EC8F381
:100ED0006F5FA8F30895EADF8D939D930895CF93F4
:100EE000CFB7CF93DF93C395869BE9F7869B0BC063
:100EF000869B09C0869B07C0869B05C0869B03C056
:100F0000869B01C08BC06F93C0918D00DD27CC56AE
:100F1000DF4F2F9365E5869B03C02F916F91E6CF3E
:100F20000F931F934F9320E040E15F9300B304744D
:100F300006FB27F93F9350E03BE039C0147440644E
:100F40002F77012F5F5F1EC0406810B314742F7796
:100F500052501FC0406400B32F770474D1F15F5F1B
:100F600000C023C0406210B32F77147491F15F5F0B
:100F700000C025C004741027515012F45D5F0000BA
:100F8000115027952C3F10B3C8F614740127015057
:100F900027952C3FC8F64227499300B304741027C5
:100FA0004F73115027952C3FA8F64695469510B3E0
:100FB000147479F00127015027952C3F98F66B5A4D
:100FC00060F3315000B3B0F600C010E41ABF002740
:100FD00019C03B503195C31BD04010E41ABF0881A3
:100FE000033C09F10B34F9F020918B001981110FAA
:100FF0001213EDCF4A81441F093651F10D3211F021
:10100000013E29F7009392003F915F914F911F910C
:101010000F912F916F91CAB7C6FD65CFDF91CF9128
:10102000CFBFCF91189520919200222369F31091A0
:101030009000112391F5343092F130939000209379
:101040008C0010918D003BE0311B30938D0027C048
:101050000091900001300CF50AE54F7049F4309191
:10106000610034FD1DC000936100C4E7D0E01CC0E6
:1010700030917F0034FD14C000937F00C0E8D0E0C1
:1010800013C0052710E000C0000002BB1AC00527EE
:1010900010E0221F1DC010E021C04AE502C032ED61
:1010A000432FC4E1D0E032E011B31464969A02B346
:1010B00011BB54E420E865E320FF052702BB279518
:1010C00017951C3FF0F66695B8F7B1F720FF052796
:1010D00002BB279517951C3FD0F62795179517FF4C
:1010E000052700001C3F02BBB0F629913A9519F77D
:1010F0000B7B10919100110FC651D04002BB11F033
:1011000010938B0010E41ABF006411B31B7B402FB7
:101110004B7B54E05A95F1F702BB11BB42BB74CF35
:1011200020917F0024FF07C02091800038E823270A
:101130002093800003C02AE520937F00FC01A1E8F2
:10114000B0E081918D9380E0A938B807D1F768E0CD
:1011500081E890E0C0DE8CE080937F000895FC0180
:1011600088E0DF011D928A95E9F708958091620079
:10117000909163000196C9F088B392E0892788BBFB
:101180008091600080FF02C0939A01C09398809183
:10119000600081FF02C0959A01C09598809160001F
:1011A00082FF02C0C09A0895C09808951F93CF93FC
:1011B000DF93CDB7DEB760970FB6F894DEBF0FBEF2
:1011C000CDBF182FCE010996CADF103211F48CE280
:1011D00044C01A3011F488E240C0193011F48BE297
:1011E0003CC0812F81568A3110F41D550DC0812FCE
:1011F00081548A3120F482E089871D5305C0812FF4
:101200008153893018F413511B8728C0103311F40F
:1012100087E223C0103421F482E089878FE11DC06A
:101220001A3321F482E0898783E317C01C3211F45A
:1012300086E313C01F3211F484E50FC01A3211F493
:1012400085E50BC01B3211F487E507C01D3211F490
:1012500086E503C01E3211F487E38B8788E0FE0128
:101260003996DE01119601900D928A95E1F7298158
:101270003A814B815C816D817E818F8198856096FA
:101280000FB6F894DEBF0FBECDBFDF91CF911F9197
:101290000895CF93DF93CDB7DEB760970FB6F8947C
:1012A000DEBF0FBECDBF8FEF81DF29873A874B8727
:1012B0005C876D877E878F87988B88E0FE013996E3
:1012C000DE01119601900D928A95E1F729813A810C
:1012D0004B815C816D817E818F81988560960FB690
:1012E000F894DEBF0FBECDBFDF91CF910895CF93AD
:1012F000DF93CDB7DEB760970FB6F894DEBF0FBEB1
:10130000CDBF2FE088E190E00FB6F894A89581BD9D
:101310000FBE21BD85B7836085BF8BB780648BBF4F
:101320008BE4809380008AE580937F008E9AA89555
:101330008B9A8D9AB89AB99A97988F98979A2FEF17
:1013400083EC99E0215080409040E1F700C000001C
:10135000A8958E987894A89580919000835087FDE9
:10136000EFC090918D000CE010E0091B11090C56A4
:101370001F4F90918C009D3209F0D1C0883009F048
:10138000DDC083EC809374008AE580936100109245
:101390006B00F8018081807661F1803241F58181B6
:1013A0008230C9F018F4813011F505C0893061F040
:1013B0008A30E9F418C08CE690E090938F00809317
:1013C0008E00CDDE28E0A0C0F801868197810197CC
:1013D00071F42FEF91C08AE690E090938F00809394
:1013E0008E0021E091C0F801838180936A0020E0A3
:1013F0008BC0F801928110927D008181811106C01D
:1014000010927E008DE790E022E070C0853019F4E4
:101410009093910068C0863009F04FC0F801838135
:10142000813041F487E89CE090938F0080938E0098
:1014300022E13FC0823041F485E69CE090938F002A
:1014400080938E0022E235C08330F1F4911108C000
:1014500085E09DE090938F0080938E0024E029C06A
:10146000913041F483EB9CE090938F0080938E0049
:1014700022E51FC09230E1F489E99CE090938F004F
:1014800080938E002AE115C0813241F487E79CE009
:1014900090938F0080938E0029E00BC0823241F43C
:1014A00086E29CE090938F0080938E002FE301C032
:1014B00020E080E480936B001DC0883069F08930A3
:1014C00019F4909393000FC08A3049F08B3059F48F
:1014D0008BE48093800007C083E990E002C08DE731
:1014E00090E021E003C08DE790E020E090938F0032
:1014F00080938E002F3F41F4F801808187FD268183
:1015000080E880936B0008C0F8018781811104C0D6
:101510008681821708F4282F209364000FC08091E1
:101520006B0087FF0BC0F8018081909160008917E4
:1015300019F0809360001ADE1092640010929000FF
:101540008091610084FF43C0809164008F3F09F463
:101550003EC0182F893008F018E0811B809364008A
:101560008091740098E8892780937400112319F101
:10157000E0918E00F0918F0080916B0086FF0BC090
:10158000A5E7B0E084918D93319685E790E0810FD7
:101590008A13F8CF0CC0CF01A5E7B0E0FC01219180
:1015A000CF012D9325E730E0210F2A13F7CFF093D9
:1015B0008F00E0938E00612F85E790E08CDC1C5F4C
:1015C0001C3019F08FEF809364001093610084E168
:1015D00090B3947431F48150D9F710929100109225
:1015E0008B0080917F0084FFACC08091620090915D
:1015F00063000196C1F5C0906600D0906700E0904E
:101600006800F090690020EAC21626E8D20621E0C0
:10161000E206F104D8F4C701B60122E03DE040E063
:1016200050E0AFD0672B682B692B81F488B392E030
:10163000892788BB82B398E0892782BB82B390E276
:10164000892782BB88B391E0892788BB80EAC816C6
:1016500086E8D80681E0E806F10428F010926300DD
:101660001092620083DDE0906200F09063008701D9
:1016700016950795093691E0190708F05BC0E0FE62
:1016800016C007DE29873A874B875C876D877E8780
:101690008F87988B88E0FE013996DE0111960190C4
:1016A0000D928A95E1F7EFEFEE1AFE0A3BC08091AA
:1016B0006A00F4E08F9FC00111248233910510F479
:1016C00082E390E04AE0489F9001499F300D112449
:1016D000442737FD4095542F609166007091670054
:1016E00080916800909169004CD0672B682B692B22
:1016F00041F5F801E75FF24F849158DD29873A8779
:101700004B875C876D877E878F87988B88E0FE018B
:101710003996DE01119601900D928A95E1F72FEF2F
:10172000E21AF20AF0926300E0926200CE010196A2
:10173000F7DC07C0879905C0109263001092620021
:1017400015DD8091660090916700A0916800B091CE
:1017500069000196A11DB11DB7FF04C0B695A795FC
:10176000979587958093660090936700A093680093
:10177000B09369008FE891E00197F1F700C0000095
:10178000EACDA1E21A2EAA1BBB1BFD010DC0AA1FA8
:10179000BB1FEE1FFF1FA217B307E407F50720F0DA
:1017A000A21BB30BE40BF50B661F771F881F991F55
:1017B0001A9469F760957095809590959B01AC019E
:1017C000BD01CF010895F894FFCFFF5AFFFFFF003E
:1017D000FFFFFFFFFFFFFFFFFFFFFFFFFFFFFFFF19
:1017E000FFFFFFFFFFFFFFFFFFFFFFFFFFFFFFFF09
:1017F000FFFFFFFFFFFFFFFFFFFFFFFFFFFF0000F7
:1018000075C0A9C08EC08DC08CC08BC08AC089C075
:1018100088C087C086C085C084C083C082C081C0A4
:1018200080C07FC07EC07E3FF9F76536F9F7593A30
:10183000F9F74038F9F7EC2DFD2DB7B6B0FCFDCF28
:1018400027BFE895B7B6B0FCFDCF21E1B7B6B6FC2F
:10185000F4CF08953230313330353037205553428C
:101860006173704C6F616465722076302E39362E4C
:1018700032206279205374657068616E2042616520
:1018800072776F6C6620286D617472697873746FFB
:10189000726D40676D782E6465290902120001019E
:1018A0000080320904000000000000001201100155
:1018B000FF000008C016DC050201010200010E0352
:1018C0005500530042006100730070001C03770054
:1018D000770077002E0066006900730063006800DF
:1018E0006C002E00640065000403090411241FBE6F
:1018F000CFE5D4E0DEBFCDBF10E0A0E6B0E0E8EF7A
:10190000FFE102C005900D92A836B107D9F720E09B
:10191000A8E6B0E001C01D92AC39B207E1F779D179
:1019200069C36ECFA82FB92F80E090E041E050EA64
:10193000609530E009C02D9182279795879510F02A
:1019400084279527305EC8F36F5FA8F30895EADF18
:101950008D939D930895CF93CFB7CF93DF93C39586
:10196000869BE9F7869B0BC0869B09C0869B07C0B8
:10197000869B05C0869B03C0869B01C089C06F9370
:10198000C0917F00DD27CA57DF4F2F9365E5869B07
:1019900003C02F916F91E6CF0F931F934F9320E0D9
:1019A00040E15F9300B3047406FB27F93F9350E0D6
:1019B0003BE039C0147440642F77012F5F5F1EC075
:1019C000406810B314742F7752501FC0406400B3A6
:1019D0002F770474D1F15F5F00C023C0406210B361
:1019E0002F77147491F15F5F00C025C00474102735
:1019F000515012F45D5F0000115027952C3F10B339
:101A0000C8F614740127015027952C3FC8F64227C9
:101A1000499300B3047410274F73115027952C3F3E
:101A2000A8F64695469510B3147479F00127015035
:101A300027952C3F98F66B5A60F3315000B3B0F6FF
:101A400000C010E41ABF002717C03B503195C31BDC
:101A5000D04010E41ABF0881033CF9F00B34E9F0E0
:101A600020917D001981110F1213EDCF093651F12C
:101A70000D3211F0013E39F7009384003F915F91E0
:101A80004F911F910F912F916F91CAB7C6FD67CFEC
:101A9000DF91CF91CFBFCF91189520918400222361
:101AA00069F310918200112339F534303AF1309303
:101AB000820020937E0010917F003BE0311B309329
:101AC0007F001CC0009182000130B4F40AE530911F
:101AD000610034FD14C000936100C2E7D0E013C080
:101AE000052710E000C0000002BB1AC0052710E067
:101AF000221F1DC010E021C04AE502C032ED432F75
:101B0000C4E1D0E032E011B31464969A02B311BB81
:101B100054E420E865E320FF052702BB27951795CD
:101B20001C3FF0F66695B8F7B1F720FF052702BB1A
:101B3000279517951C3FD0F62795179517FF052772
:101B400000001C3F02BBB0F629913A9519F70B7BB8
:101B500010918300110FC651D04002BB11F01093B9
:101B60007D0010E41ABF006411B31B7B402F4B7B38
:101B700054E05A95F1F702BB11BB42BB7FCFF894FA
:101B80008E9A97981BBE15BEF1E0FBBF1BBE38C2F4
:101B900031978040E9F70895FC013381932F448108
:101BA000842F2281203339F44370E42FF0E0ED5983
:101BB000FF4F80810895283529F431110EC0E1E0EE
:101BC000F0E006C0203571F4311121C0E0E0F0E012
:101BD00089E080935700849108953830C1F4E3E0A0
:101BE000F0E0F6CF203221F4FC01EE0FFF1F06C01B
:101BF000283231F4FC01EE0FFF1F319684910895D5
:101C0000203A09F4E2C1203C11F46581E6D180E07C
:101C1000089511BA80E882BB14BE81E08BBF82E0D8
:101C20008BBF84E0B5DF8799AADF85B7826085BF67
:101C30008BB780648BBF8E9A80E1AADF8E987894F0
:101C400080918200835087FD2DC190917F00CCE070
:101C5000D0E0C91BD109CA57DF4F90917E009D3259
:101C600009F0B7C0883009F01BC183EC8093720083
:101C70008AE58093610010926800888180762981CE
:101C80008823B9F189E690E09093810080938000E9
:101C9000233031F4CE0180DF80936C0024E08FC0CC
:101CA000253019F12A3009F1822F8450863098F4BA
:101CB0008A819B8190936E0080936D002930B9F0EA
:101CC0008E8180936F008D8182708093700020934D
:101CD00071002FEF6DC080916000223011F48E7F73
:101CE00001C081608093600002C021E068C020E0F4
:101CF00066C08A8110927B00211106C010927C0080
:101D00008BE790E022E04EC0253019F480938300E9
:101D10003DC02630A9F59B81913019F48CEA98E1F9
:101D200004C0923041F48AE998E190938100809355
:101D3000800022E121C09330F1F4811108C088EEC7
:101D400098E1909381008093800024E015C0813059
:101D500041F48CEC98E190938100809380002CE119
:101D60000BC0823041F48EEB98E190938100809318
:101D700080002EE001C020E080E48093680016C05F
:101D8000283069F0293029F4809385008BE790E0B2
:101D900004C08BE790E02A3021F020E003C085E802
:101DA00090E021E090938100809380002F3F39F4F0
:101DB000888187FD2E8180E88093680007C08F812D
:101DC000811104C08E81821708F4282F20936200AD
:101DD00067C09091680097FF63C090916F00F82EE4
:101DE000981708F4F92E9F1990936F00EE24E3944E
:101DF0009111E12C809171008730B0F08E010FC0FD
:101E0000D8016D918D0180916D0090916E009C01C3
:101E10002F5F3F4F30936E0020936D00DED0802FF8
:101E20008C1B8F1568F339C080917000E0916D00B4
:101E3000F0916E009F2DDE0190FD9395925048F138
:101E4000F83138F522D0F8940D901D9021E017D08C
:101E50002E2F2E5F2F7331F0EE2079F0882369F05A
:101E6000903059F423E00BD010D025E008D00DD0ED
:101E700007B606FE02C021E102D03296DFCFF89409
:101E800027BFE89511247894089507B600FCFDCF8C
:101E90000895F0936E00E0936D00E11010926200DF
:101EA000109282008091610084FF73C08091620073
:101EB0008F3F09F46EC0F82E893010F028E0F22E22
:101EC0008F19809362008091720098E8892780932F
:101ED0007200FF2009F44BC08091680087FF28C082
:101EE00080916F008F1508F4F82E8F1980936F0082
:101EF000E0907100C3E7D0E014C000916D00109134
:101F00006E00A6E0AE1518F4C8015FD002C0F8015B
:101F10008491888321960F5F1F4F10936E0000936A
:101F20006D0083E790E0FC2FF81BFF1530F31CC019
:101F3000E0918000F0918100A3E7B0E086FF09C046
:101F400084918D93319683E790E08F0D8A13F8CFBB
:101F500007C081918D9383E790E08F0D8A13F9CFAD
:101F6000F0938100E093800028E02F1560F06F2D42
:101F700083E790E0ECDC8F2D8C5F8C3041F09FEF9D
:101F80009093620004C08FEF809362008EE1809393
:101F9000610084E190B3947431F48150D9F71092C8
:101FA000830010927D0080916000803118F0879945
:101FB000805104C0823010F0879B82508093600073
:101FC0008091600081113CCE2FCEE199FECF9FBB66
:101FD0008EBBE09A99278DB30895262FE199FECF05
:101FE0009FBB8EBB2DBB0FB6F894E29AE19A0FBE51
:101FF00001960895F894FFCFFE5AFF1E9307000044
:00000001FF
